:020000040000FA
:0600000048EF31F0120090
:0600080004EF08F01200F5
:060018000CEF08F01200DD
:0610000048EF31F0120080
:061008008FEF29F0120039
:0610180098EF29F0120020
:06102A000200C06200009C
:101030009200000021000000BA620000CC00000015
:0410400006000000A6
:0C104400D9CFE6FFE1CFD9FFFB0EDB5057
:1010500029E10201BB51EA6A000FE96E010EEA22A2
:101060003C0EEF6EBB29EA6A000FE96E010EEA2220
:10107000FE0EDBCFEFFF020EBB25EA6A000FE96E22
:10108000010EEA22FD0EDBCFEFFF030EBB25EA6A5D
:10109000000FE96E010EEA22FC0EDBCFEFFF040E1B
:1010A000BB273BD00201BB51EA6A000FE96E010E7B
:1010B000EA223C0EEF6EBB29EA6A000FE96E010ED0
:1010C000EA22FE0EDBCFEFFF020EBB25EA6A000F1D
:1010D000E96E010EEA22FD0EDBCFEFFF030EBB250A
:1010E000EA6A000FE96E010EEA22FC0EDBCFEFFF89
:1010F000040EBB25EA6A000FE96E010EEA22FB0E20
:10110000DBCFEFFF050EBB25EA6A000FE96E010E8B
:10111000EA223A0EEF6E060EBB27E552E7CFD9FF63
:101120001200D9CFE6FFE1CFD9FFFE0EDB50410818
:1011300020E1FD0EDB50350A18E0060A13E0010A33
:101140000EE0030A09E0010A04E00001CA0E956FEF
:101150000FD0010EC26E0CD0050EC26E09D0090E62
:10116000C26E06D00D0EC26E03D0110EC26E00D03C
:101170000FD0FE0EDB5042080BE1FD0EDB50320AB1
:1011800004E00001CA0E956F03D0210EC26E00D09C
:10119000E552E7CFD9FF1200D9CFE6FFE1CFD9FF63
:1011A000FE0EDBCFE9FFEA6AE9BEEA688B0EE926AC
:1011B000000EEA22EF50690A1DE00C0A18E0010A4D
:1011C00013E0070A0EE0010A09E0030A04E0000147
:1011D000CA0E956F12D0010EC26E0FD0050EC26EF0
:1011E0000CD0090EC26E09D00D0EC26E06D0110EC3
:1011F000C26E03D0210EC26E00D0E552E7CFD9FFF8
:101200001200D9CFE6FFE1CFD9FFE652DF6A060E22
:10121000DF24EA6A600FE96E000EEA22EF50E66E04
:10122000DF50EA6A8B0FE96E000EEA22E552E750C2
:10123000EF6EDFCFE6FFB0DFE552DF2A060EDF24D8
:10124000EA6A600FE96E000EEA22EF50290803E017
:10125000070EDF5CDCE3060EDF24EA6A600FE96E4E
:10126000000EEA22EF5029080CE1070EDF5C09E2CC
:10127000DF50EA6A8B0FE96E000EEA22290EEF6E4C
:1012800003D00001CC0E956FE552E552E7CFD9FFB0
:101290001200D9CFE6FFE1CFD9FF030EE126FD0E04
:1012A000DB500F0BDF6EFD0EDB380F0B0F0BE76E05
:1012B000010EE7CFDBFFFD0EDBCF14F0FE0EDBCF20
:1012C00015F015C014F0156A0F0E1414E76E020E17
:1012D000E7CFDBFFDF50090805E2370EDF2400010E
:1012E000D26F04D0300EDF240001D26F010EDB502C
:1012F000090805E2010EDB50370FD36F04D0010E51
:10130000DB50300FD36F020EDB50090805E2020EEE
:10131000DB50370FD46F04D0020EDB50300FD46F88
:10132000FB0EDBCFE9FFEA6AE9BEEA687F0EE92639
:10133000020EEA22FC0EDBCFEFFFFB0EDB28E96E8C
:10134000EA6AE9BEEA687F0EE926020EEA22300E5A
:10135000EF6EFB0EDB50020FE96EEA6AE9BEEA6847
:101360007F0EE926020EEA22D4C0EFFFFB0EDB500F
:10137000030FE96EEA6AE9BEEA687F0EE926020E0B
:10138000EA22D3C0EFFFFB0EDB50040FE96EEA6ADE
:10139000E9BEEA687F0EE926020EEA22D2C0EFFF1C
:1013A000FB0EDB50050FE96EEA6AE9BEEA687F0EC4
:1013B000E926020EEA227C0EEF6E030EE15C02E2E9
:1013C000E16AE552E16EE552E7CFD9FF1200D9CFCD
:1013D000E6FFE1CFD9FFFE0EDB50410828E1780E91
:1013E000E66EE66E8050200B01E0010E300FE66ED7
:1013F000780EE66E8050080B01E0010E300FE66EAD
:101400008050040B01E0010E300FE66E8050020B9D
:1014100001E0010E300FE66E8050010B300FE66EDA
:1014200009EC25F0146E080EE15E145056D0FE0E45
:10143000DB50420828E1780EE66EE66E8150200B04
:1014400001E0010E300FE66E8150100B01E0010E3D
:10145000300FE66E780EE66E8150040B01E0010E4F
:10146000300FE66E8150020B01E0010E300FE66E88
:101470008150010B300FE66E09EC25F0146E080E5A
:10148000E15E14502AD0FE0EDB50430826E1825064
:10149000800B01E0010E300FE66E8250400B01E040
:1014A000010E300FE66E780EE66EE66EE66E825046
:1014B000040B01E0010E300FE66E8250020B01E0DA
:1014C000010E300FE66E8250010B300FE66E09EC14
:1014D00025F0146E080EE15E1450E552E7CFD9FFF7
:1014E0001200D9CFE6FFE1CFD9FFFE0EDB50410855
:1014F00001E0D2D0FD0EDB50350A01E1A5D0060A8D
:1015000001E17BD0010A52E0030A29E0010A01E06F
:10151000C2D0FC0EDB50300802E180901FD0FC0EE0
:10152000DB50310802E1808019D0FC0EDB506908E5
:1015300007E19280C1500E0802E30F0EC16E0ED07B
:10154000FC0EDB506F0803E19290809007D0FC0EF8
:10155000DB50610803E192800E0EC16E9CD0FC0E40
:10156000DB50300802E1809220D0FC0EDB503108C5
:1015700002E180821AD0FC0EDB50690807E19282FA
:10158000C1500D0802E30E0EC16E0FD0FC0EDB50F1
:101590006F0803E19292809208D0FC0EDB50610844
:1015A00004E1030E92120D0EC16E75D0FC0EDB50DD
:1015B000300802E1809420D0FC0EDB50310802E1BB
:1015C00080841AD0FC0EDB50690807E19284C15078
:1015D0000C0802E30D0EC16E0FD0FC0EDB506F083D
:1015E00003E19294809408D0FC0EDB50610804E182
:1015F000070E92120C0EC16E4ED0FC0EDB5030085E
:1016000002E1809620D0FC0EDB50310802E180869A
:101610001AD0FC0EDB50690807E19286C1500B0816
:1016200002E30C0EC16E0FD0FC0EDB506F0803E11D
:101630009296809608D0FC0EDB50610804E10F0EF4
:1016400092120B0EC16E27D0FC0EDB50300802E167
:10165000809A20D0FC0EDB50310802E1808A1AD03B
:10166000FC0EDB50690807E1928AC1500A0802E3C8
:101670000B0EC16E0FD0FC0EDB506F0803E1929A87
:10168000809A08D0FC0EDB50610804E12F0E921204
:101690000A0EC16E00D013D1FE0EDB50420801E0ED
:1016A0007FD0FD0EDB50350A6EE0010A60E0060ACD
:1016B00037E0030A1CE0010A01E071D0FC0EDB50A8
:1016C000300802E1819012D0FC0EDB50310802E1BB
:1016D00081800CD0FC0EDB50690802E1938006D0BB
:1016E000FC0EDB506F0802E19390819058D0FC0E05
:1016F000DB50300802E1819212D0FC0EDB50310841
:1017000002E181820CD0FC0EDB50690802E1938279
:1017100006D0FC0EDB506F0802E1939281923FD01D
:10172000FC0EDB50300802E1819420D0FC0EDB502F
:10173000310802E181841AD0FC0EDB50690807E110
:101740009384C150060802E30A0EC16E0FD0FC0E4E
:10175000DB506F0803E19394819408D0FC0EDB50BA
:10176000610804E192689384060EC16E18D0FC0EE5
:10177000DB50300802E1819805D0FC0EDB503108C7
:1017800001E181880CD0FC0EDB50300802E1819A27
:1017900005D0FC0EDB50310801E1818A00D08FD0EA
:1017A000FE0EDB50430801E08AD0FD0EDB50370A05
:1017B0006DE0010A52E0040A37E0030A1CE0010A66
:1017C00001E07DD0FC0EDB50300802E1829012D0A7
:1017D000FC0EDB50310802E182800CD0FC0EDB50A5
:1017E000690802E1948006D0FC0EDB506F0802E12C
:1017F0009490829064D0FC0EDB50300802E182921B
:1018000012D0FC0EDB50310802E182820CD0FC0EBB
:10181000DB50690802E1948206D0FC0EDB506F08B1
:1018200002E1949282924BD0FC0EDB50300802E130
:10183000829412D0FC0EDB50310802E182840CD07D
:10184000FC0EDB50690802E1948406D0FC0EDB50EC
:101850006F0802E19494829432D0FC0EDB50300881
:1018600002E1829C12D0FC0EDB50310802E1828C36
:101870000CD0FC0EDB50690802E1948C06D0FC0E03
:10188000DB506F0802E1949C829C19D0FC0EDB5067
:10189000300802E1829E12D0FC0EDB50310802E1DA
:1018A000828E0CD0FC0EDB50690802E1948E06D0CB
:1018B000FC0EDB506F0802E1949E829E00D0E55240
:1018C000E7CFD9FF1200D9CFE6FFE1CFD9FF020E53
:1018D000E126FE0EDB500F0BDF6EFE0EDB380F0B2A
:1018E0000F0BE76E010EE7CFDBFFDF50090805E2C3
:1018F000370EDF240001D26F04D0300EDF24000148
:10190000D26F010EDB50090805E2010EDB50370FE4
:10191000D36F04D0010EDB50300FD36FFC0EDBCF42
:10192000E9FFEA6AE9BEEA687F0EE926020EEA22CA
:10193000FD0EDBCFEFFFFC0EDB28E96EEA6AE9BEA5
:10194000EA687F0EE926020EEA22780EEF6EFC0EA0
:10195000DB50020FE96EEA6AE9BEEA687F0EE9260B
:10196000020EEA22780EEF6EFC0EDB50030FE96EDA
:10197000EA6AE9BEEA687F0EE926020EEA22D3C0CF
:10198000EFFFFC0EDB50040FE96EEA6AE9BEEA687D
:101990007F0EE926020EEA22D2C0EFFFFC0EDB50DA
:1019A000050FE96EEA6AE9BEEA687F0EE926020ED3
:1019B000EA227C0EEF6E020EE15C02E2E16AE55281
:1019C000E16EE552E7CFD9FF1200D9CFE6FFE1CFB4
:1019D000D9FFFD0EDB50650810E1FE0EDB50320A28
:1019E00007E0030A01E008D094940C0EBD6E04D009
:1019F00094920C0EBA6E00D011D0FD0EDB5064082C
:101A00000DE1FE0EDB50320A06E0030A01E006D0CB
:101A1000BD6A948403D0BA6A948200D0E552E7CFBD
:101A2000D9FF1200D9CFE6FFE1CFD9FFCB50146E1A
:101A3000156A166A176A142A000E15221622172232
:101A400014C006F015C007F016C008F017C009F062
:101A5000FA0EDBCF0BF0FB0EDBCF0CF0FC0EDBCF76
:101A60000DF0FD0EDBCF0EF09CEC2FF002C006F067
:101A700003C007F004C008F005C009F00B6A010EAE
:101A80000C6E0D6A0E6A51EC2EF0FA0E06C0DBFFEA
:101A9000FB0E07C0DBFFFC0E08C0DBFFFD0E09C01C
:101AA000DBFFFE0EDB50320A0EE0030A01E016D027
:101AB000FA0EDBCFE6FFFB0EDBCFE6FF03EC30F0E8
:101AC000E552E5520BD0FA0EDBCFE6FFFB0EDBCF83
:101AD000E6FFD4EC2FF0E552E55200D0E552E7CF17
:101AE000D9FF1200D9CFE6FFE1CFD9FFFD0EDBCF42
:101AF00014F0FE0EDBCF15F0D890155004E62F0E33
:101B0000145C000E15581FE3E00E086E2E0E096ED1
:101B1000FD0EDBCF0DF0FE0EDBCF0EF0FEEC2DF058
:101B200008C014F009C015F01406000E155AFD0E79
:101B300014C0DBFFFE0E15C0DBFF040EE66E07ECE3
:101B400031F0E55275D0FD0EDBCF14F0FE0EDBCF89
:101B500015F0D890155004E60C0E145C000E1558C4
:101B60002CE3FD0EDBCF16F0FE0EDBCF17F01734A3
:101B700004E216502E08000E17541FE3B80E086E2C
:101B80000B0E096EFD0EDBCF0DF0FE0EDBCF0EF05F
:101B9000FEEC2DF008C014F009C015F01406000E7C
:101BA000155AFD0E14C0DBFFFE0E15C0DBFF050E3F
:101BB000E66E07EC31F0E5523BD0FD0EDBCF14F0C2
:101BC000FE0EDBCF15F0D890155004E6030E145C22
:101BD000000E15582CE3FD0EDBCF16F0FE0EDBCF0A
:101BE00017F0173404E216500B08000E17541FE3C9
:101BF000EE0E086E020E096EFD0EDBCF0DF0FE0E2E
:101C0000DBCF0EF0FEEC2DF008C014F009C015F08B
:101C10001406000E155AFD0E14C0DBFFFE0E15C093
:101C2000DBFF060EE66E07EC31F0E55201D0CB6A21
:101C3000FD0EDB50CB6EE552E7CFD9FF1200D9CFB6
:101C4000E6FFE1CFD9FFFE0EDB50380A3EE00F0A77
:101C500036E0010A2EE0030A26E0010A1EE0070A28
:101C600016E0010A0EE0030A06E0010A01E033D0A3
:101C700059EC31F030D0100EE66EEBEC30F0E5525E
:101C80002AD0110EE66EEBEC30F0E55224D0120EA5
:101C9000E66EEBEC30F0E5521ED0130EE66EEBEC88
:101CA00030F0E55218D0140EE66EEBEC30F0E55251
:101CB00012D0150EE66EEBEC30F0E5520CD0160E9D
:101CC000E66EEBEC30F0E55206D0170EE66EEBEC6C
:101CD00030F0E55200D0E552E7CFD9FF1200D9CF5E
:101CE000E6FFE1CFD9FF060EE126DE6ADE6ADE6A94
:101CF000DD6ADD52DD52040EDB6A050EDB6AFD0E85
:101D0000DBCF14F0FE0EDBCF15F0166A176A15AEA6
:101D100002D01668176814C0DFFF010E15C0DBFF84
:101D2000020E16C0DBFF030E17C0DBFFFC0EDB50FC
:101D30006D0801E0AFD100018A97FD0EDBCF17F0EF
:101D4000FE0EDBCF18F0196A18BE1968600E146E0B
:101D5000EA0E156E166A14C007F015C008F016C01A
:101D600009F017C00CF018C00DF019C00EF024ECEB
:101D70002EF007C0A7F008C0A8F0FD0EDBCF14F0CE
:101D8000FE0EDBCF15F0153404E21450F408010EFA
:101D9000155441E2FD0EDBCF16F0FE0EDBCF17F03F
:101DA000173404E21650E708030E175434E3170EF5
:101DB000E66EEBEC30F0E552D9CFE9FFDACFEAFF7F
:101DC000EECF06F0EECF07F0EECF08F0EFCF09F040
:101DD0001B0E0B6EB70E0C6E0D6A0E6A9CEC2FF08C
:101DE00002C006F003C007F004C008F005C009F007
:101DF000E80E0B6E030E0C6E0D6A0E6A32EC30F0BC
:101E000006C0DEFF07C0DEFF08C0DEFF09C0DDFF41
:101E1000DD52DD5209D1FD0EDBCF14F0FE0EDBCF1B
:101E200015F0153404E214506408000E155442E213
:101E3000FD0EDBCF16F0FE0EDBCF17F0173404E2F9
:101E40001650F408010E175435E3160EE66EEBEC4F
:101E500030F0E552D9CFE9FFDACFEAFFEECF06F056
:101E6000EECF07F0EECF08F0EFCF09F0360E0B6E95
:101E70006E0E0C6E010E0D6E0E6A9CEC2FF002C001
:101E800006F003C007F004C008F005C009F0E80E32
:101E90000B6E030E0C6E0D6A0E6A32EC30F006C04B
:101EA000DEFF07C0DEFF08C0DEFF09C0DDFFDD5238
:101EB000DD52BAD0FD0EDBCF14F0FE0EDBCF15F0F5
:101EC000153404E214503208000E155431E2FD0EB0
:101ED000DBCF16F0FE0EDBCF17F0173404E21650FE
:101EE0006408000E175424E3140EE66EEBEC30F099
:101EF000E552D9CFE9FFDACFEAFFEECF06F0EECF19
:101F000007F0EECF08F0EFCF09F0770E0B6E010E61
:101F10000C6E0D6A0E6A9CEC2FF002C0DEFF03C04F
:101F2000DEFF04C0DEFF05C0DDFFDD52DD527CD0E8
:101F3000FD0EDBCF14F0FE0EDBCF15F0153404E2FE
:101F400014500A08000E155431E2FD0EDBCF16F0D6
:101F5000FE0EDBCF17F0173404E216503208000EE5
:101F6000175424E3130EE66EEBEC30F0E552D9CFB4
:101F7000E9FFDACFEAFFEECF06F0EECF07F0EECFC3
:101F800008F0EFCF09F0EE0E0B6E020E0C6E0D6A2C
:101F90000E6A9CEC2FF002C0DEFF03C0DEFF04C01F
:101FA000DEFF05C0DDFFDD52DD523ED0FD0EDBCF92
:101FB00014F0FE0EDBCF15F0D890155004E6010E9C
:101FC000145C000E155830E3FD0EDBCF16F0FE0E4C
:101FD000DBCF17F0173404E216500A08000E17542E
:101FE00023E3100EE66EEBEC30F0E552D9CFE9FFBB
:101FF000DACFEAFFEECF06F0EECF07F0EECF08F033
:10200000EFCF09F0700E0B6E170E0C6E0D6A0E6A94
:102010009CEC2FF002C0DEFF03C0DEFF04C0DEFF39
:1020200005C0DDFFDD52DD52176A186A010E196E18
:10203000DFCF1AF0DBCF1BF01C6A1BBE1C681A50E6
:10204000175C146E1B501858156E1C501958166EDC
:10205000190E1426000E15221622040E14C0DBFFE2
:10206000050E15C0DBFFF294040EDBCFE6FF050E74
:10207000DBCFE6FFCFEC30F0E552E552040EDBCFCC
:1020800014F0050EDBCF15F014C0F3FF15C0F4FFFC
:102090009ED09DD0FC0EDB50750801E095D000016C
:1020A0008A870001E80EA96F030EAA6FFD0EDBCF31
:1020B00017F0FE0EDBCF18F0196A18BE1968600E13
:1020C000146EEA0E156E166A14C007F015C008F0FB
:1020D00016C009F017C00CF018C00DF019C00EF0B2
:1020E00024EC2EF007C0A7F008C0A8F0FD0EDBCF4F
:1020F00014F0FE0EDBCF15F0D890155004E6010E5B
:10210000145C000E15582FE3FD0EDBCF16F0FE0E0B
:10211000DBCF17F0173404E21650E708030E17540C
:1021200022E3100EE66EEBEC30F0E552D9CFE9FF7A
:10213000DACFEAFFEECF06F0EECF07F0EECF08F0F1
:10214000EFCF09F0060E0B6E0C6A0D6A0E6A9CEC5E
:102150002FF002C0DEFF03C0DEFF04C0DEFF05C0BB
:10216000DDFFDD52DD52176A186A010E196EDFCFEE
:102170001AF0DBCF1BF01C6A1BBE1C681A50175CE0
:10218000146E1B501858156E1C501958166E040EFC
:1021900014C0DBFF050E15C0DBFFF294040EDBCF8D
:1021A000E6FF050EDBCFE6FFCFEC30F0E552E5525F
:1021B000040EDBCF14F0050EDBCF15F014C0F3FFD7
:1021C00015C0F4FF04D003D00001CB0E956F060EAE
:1021D000E15C02E2E16AE552E16EE552E7CFD9FF48
:1021E0001200D9CFE6FFE1CFD9FFFE0EDB50340A53
:1021F0001EE0070A16E0010A0EE0030A06E0010AE3
:1022000001E01BD056EC31F018D04D0EE66E56ECC6
:1022100030F0E55212D05D0EE66E56EC30F0E5522D
:102220000CD06D0EE66E56EC30F0E55206D07D0E09
:10223000E66E56EC30F0E55200D0E552E7CFD9FF1C
:102240001200D9CFE6FFE1CFD9FF060EE126DE6A04
:10225000DE6ADE6ADD6ADD52DD52040EDB6A050EDF
:10226000DB6AFD0EDBCF14F0FE0EDBCF15F0166A35
:10227000176A15AE02D01668176814C0DFFF010E8A
:1022800015C0DBFF020E16C0DBFF030E17C0DBFF1D
:10229000FC0EDB506D0801E029D1FD0EDBCF14F000
:1022A000FE0EDBCF15F0153404E214501408000EB6
:1022B000155431E2FD0EDBCF16F0FE0EDBCF17F02A
:1022C000173404E216502808000E175424E37D0E3C
:1022D000E66E56EC30F0E552D9CFE9FFDACFEAFFEF
:1022E000EECF06F0EECF07F0EECF08F0EFCF09F01B
:1022F000DC0E0B6E050E0C6E0D6A0E6A9CEC2FF058
:1023000002C0DEFF03C0DEFF04C0DEFF05C0DDFF4C
:10231000DD52DD52BAD0FD0EDBCF14F0FE0EDBCF66
:1023200015F0153404E214500A08000E155431E279
:10233000FD0EDBCF16F0FE0EDBCF17F0173404E2F4
:1023400016501408000E175424E36D0EE66E56EC7A
:1023500030F0E552D9CFE9FFDACFEAFFEECF06F051
:10236000EECF07F0EECF08F0EFCF09F0B80E0B6E0E
:102370000B0E0C6E0D6A0E6A9CEC2FF002C0DEFF95
:1023800003C0DEFF04C0DEFF05C0DDFFDD52DD520D
:102390007CD0FD0EDBCF14F0FE0EDBCF15F0153434
:1023A00004E214500508000E155431E2FD0EDBCF97
:1023B00016F0FE0EDBCF17F0173404E216500A08B1
:1023C000000E175424E35D0EE66E56EC30F0E55235
:1023D000D9CFE9FFDACFEAFFEECF06F0EECF07F074
:1023E000EECF08F0EFCF09F0700E0B6E170E0C6EEB
:1023F0000D6A0E6A9CEC2FF002C0DEFF03C0DEFF08
:1024000004C0DEFF05C0DDFFDD52DD523ED0FD0E13
:10241000DBCF14F0FE0EDBCF15F0D890155004E69C
:10242000010E145C000E155830E3FD0EDBCF16F0E4
:10243000FE0EDBCF17F0173404E216500508000E2D
:10244000175423E34D0EE66E56EC30F0E552D9CF2B
:10245000E9FFDACFEAFFEECF06F0EECF07F0EECFDE
:1024600008F0EFCF09F0E00E0B6E2E0E0C6E0D6A29
:102470000E6A9CEC2FF002C0DEFF03C0DEFF04C03A
:10248000DEFF05C0DDFFDD52DD52176A186A010E5E
:10249000196EDFCF1AF0DBCF1BF01C6A1BBE1C6865
:1024A0001A50175C146E1B501858156E1C50195892
:1024B000166E040E14C0DBFF050E15C0DBFF9E90E8
:1024C000040EDBCFE6FF050EDBCFE6FFB3EC30F00A
:1024D000E552E552040EDBCF14F0050EDBCF15F00C
:1024E00014C0F3FF15C0F4FF76D075D0FC0EDB509E
:1024F00075086EE1FD0EDBCF14F0FE0EDBCF15F09C
:10250000D890155004E6010E145C000E15582FE308
:10251000FD0EDBCF16F0FE0EDBCF17F0173404E212
:102520001650E708030E175422E34D0EE66E56ECE4
:1025300030F0E552D9CFE9FFDACFEAFFEECF06F06F
:10254000EECF07F0EECF08F0EFCF09F00C0E0B6ED8
:102550000C6A0D6A0E6A9CEC2FF002C0DEFF03C00D
:10256000DEFF04C0DEFF05C0DDFFDD52DD52176A6D
:10257000186A010E196EDFCF1AF0DBCF1BF01C6A50
:102580001BBE1C681A50175C146E1B501858156E31
:102590001C501958166E040E14C0DBFF050E15C032
:1025A000DBFF9E90040EDBCFE6FF050EDBCFE6FFE0
:1025B000B3EC30F0E552E552040EDBCF14F0050E1B
:1025C000DBCF15F014C0F3FF15C0F4FF04D003D027
:1025D0000001CB0E956F060EE15C02E2E16AE55266
:1025E000E16EE552E7CFD9FF1200D9CFE6FFE1CF88
:1025F000D9FF040EE126DF6A010EDB6A020EDB6AF8
:10260000030EDB6A5A0E0001615D1DE14D0E625D35
:1026100019E1440E635D16E1310EE66E760EE66E4C
:10262000320EE66E310EE66E500EE66E430EE66E2C
:10263000690EE66E3A0EE66E09EC25F0146E080E91
:10264000E15E1450AAD04D0E615D1BE1440E625D47
:1026500008E1490E635D05E10F0EC16E9268936853
:102660000FD0410E625D0CE14E0E635D09E1926890
:10267000040E936E010EC26E060EC16EBF0EC06ECA
:102680008CD0440E615D01E088D0500E625D2BE17C
:10269000410E635D28E1780EE66EE66E8050200BF9
:1026A00001E0010E300FE66E780EE66E8050080BEA
:1026B00001E0010E300FE66E8050040B01E0010EC8
:1026C000300FE66E8050020B01E0010E300FE66E17
:1026D0008050010B300FE66E09EC25F0146E080EE9
:1026E000E15E14505AD0500E625D2BE1420E635DE4
:1026F00028E1780EE66EE66E8150200B01E0010EB7
:10270000300FE66E8150100B01E0010E300FE66EC7
:10271000780EE66E8150040B01E0010E300FE66E7C
:102720008150020B01E0010E300FE66E8150010B6B
:10273000300FE66E09EC25F0146E080EE15E1450C1
:102740002CD0500E625D29E1430E635D26E182507C
:10275000800B01E0010E300FE66E8250400B01E06D
:10276000010E300FE66E780EE66EE66EE66E825073
:10277000040B01E0010E300FE66E8250020B01E007
:10278000010E300FE66E8250010B300FE66E09EC41
:1027900025F0146E080EE15E1450020E0001955DE6
:1027A00002E10001646B040EE15C02E2E16AE552C1
:1027B000E16EE552E7CFD9FF1200D9CFE6FFE1CFB6
:1027C000D9FFE652F250800B01E0010EDF6EF29E5F
:1027D000A69EA69CA684FE0EDB50A96EFD0EDB50C5
:1027E000A86E550EA76EAA0EA76EA682A6B2FED739
:1027F000A694DF50E8B0F28EE8A0F29EE552E552D2
:10280000E7CFD9FF1200D9CFE6FFE1CFD9FFA69CD1
:10281000A69EFE0EDB50A96EA680A85000D0E55201
:10282000E7CFD9FF1200D9CFE6FFE1CFD9FFE652BB
:10283000FB0EDB50F66EFC0EDB50F76EFD0EDB5030
:10284000F86EE00EF616DF6ADFCF14F03F0EE76E8B
:102850001418E8AE02D0143403D0E750D8801454D2
:1028600012E30900DFCF14F0156A14BE1568F90EE3
:10287000DB501424E96EFA0EDB501520EA6EF5CF1A
:10288000EFFFDF2AE1D7E552E552E7CFD9FF12008B
:10289000D9CFE6FFE1CFD9FFE652A6B2FED7F29C30
:1028A000F29EFD0EDB50F86EFC0EDB50F76EFB0E59
:1028B000DB50F66EE00EF616A68EA69CA684A688C1
:1028C000550EA76EAA0EA76EA6820000F90EDBCFEA
:1028D00014F0FA0EDBCF15F015C014F0156A145081
:1028E000EA6EFF0EE76EF90EDBCF14F0FA0EDBCFC7
:1028F00015F0E7501416156A1450E96E0A00200E00
:10290000DF6EDF5005E0EE50F56E0F00DF06F9D701
:10291000A68EA69CA684550EA76EAA0EA76EA682AA
:102920000000200EDF6EDF5005E0EE50F56E0F0068
:10293000DF06F9D7A68EA69CA684550EA76EAA0E12
:10294000A76EA6820000A694F28EF28CE552E552A4
:10295000E7CFD9FF1200550EA76EAA0EA76EA6826A
:10296000A6B2FED7A6941200D9CFE6FFE1CFD9FFD9
:10297000F29CF29EFD0EDB50F86EFC0EDB50F76E03
:10298000FB0EDB50F66E0001D76B0E0E0001D75D1B
:1029900017E20001D751E76EF90EDBCFE9FFFA0E1F
:1029A000DBCFEAFFE750E926000EEA22EF50F56E92
:1029B0000C00C40EA66ECFDF09000001D72BE5D7AF
:0C29C000F28EF28CE552E7CFD9FF120036
:0429CC00D9CFE6FF7A
:1029D000E1CFD9FFE652A09A6A6A686A706A020E6D
:1029E000E66EE66AE66A710EE66E0F0EE66E82EC41
:1029F0002FF0146E050EE15E1450160E6F6E9F0ED2
:102A00006B6E7B0E696EDF6ADF50146E156A0C0EFA
:102A1000145C000E155810E2DF50040DF3CFE9FFEF
:102A2000F4CFEAFF000EE926040EEA22EE6AEE6A0F
:102A3000EE6AEE6ADF2AE8D76D8C6E6A6D986D9C3F
:102A400068A607D068960201D96BDE6BDF6BE06B7E
:102A5000F7D70201010EF26FF36FF46BF56BE66BC3
:102A6000DF6A030EDF5C26E2EA6ADF34FE0BEA3639
:102A7000E96ECF0EE926020EEA22EE6AED6AEA6AF4
:102A8000DF34FE0BEA36E96EC90EE926020EEA22B1
:102A9000EE6AED6ADF50EA6AEA0FE96E020EEA2298
:102AA000EF6ADF50EA6AED0FE96E020EEA22EF6A82
:102AB000DF2AD7D70201080ECF6F040ED06F160E93
:102AC000706E0401300E026F040E036F080E016F6A
:102AD000840E006F0201C36BC26BE552E552E7CF73
:102AE000D9FF1200D9CFE6FFE1CFD9FFE6520201AC
:102AF000C25116E106D06D6A696A0201C26BA19AE1
:102B0000B9D06D6A696A160E6F6E9F0E6B6E7B0E82
:102B1000696E6DB602D06D86FCD70201010EC26FE0
:102B2000C20508E16DBA06D0686A696A6980698879
:102B3000020EC26F6850040B05E06950040B02E0FE
:102B40006894CBD86DA202D0A19A94D06850010BA2
:102B500008E06950010B05E039DF0201040EC26F85
:102B600068906850100B05E06950100B02E0A0D887
:102B7000689868AC19D069AC0FD0010EE66EE66AB1
:102B8000000EE66EE66A730EE66EE66A85EC2BF0E2
:102B9000146E060EE15E1450689C0201F05101E0D3
:102BA000F007F05101E165DB6850200B04E069504B
:102BB000200B01E064D86850020B13E06950020B4F
:102BC00010E0010EE66EE66A000EE66EE66AE66862
:102BD0007F0EE66E85EC2BF0146E060EE15E14504F
:102BE0006A6A040E0201E76EC219E8AE02D0E73449
:102BF00002D0E750C25D02E2A19A3CD069A639D06A
:102C0000DF6A040EDF5C35E268A630D06CCFE7F2F5
:102C10000201E751780BE842E842E842E86F689623
:102C2000E7B508D0E851EA6AED0FE96E020EEA2234
:102C3000EF7007D0E851EA6AEA0FE96E020EEA2265
:102C4000EF70E85102E160D810D0000EE66EE66A3F
:102C5000E70EE66E020EE66E720EE66EE66A85EC32
:102C60002BF0146E060EE15E145001D002D0DF2A64
:102C7000C8D7A19AE552E552E7CFD9FF120070A05C
:102C800015D0C5C2E9FFC6C2EAFFEF5080080DE1CA
:102C9000CFC2E9FFD0C2EAFFEF50840806E1C5C207
:102CA000E9FFC6C2EAFF8C0EEF6E7090689A1200C0
:102CB000698468986D820201010EE66F000EE66E6F
:102CC000E66AE66EE66A750EE66EE66A85EC2BF05D
:102CD000146E060EE15E145012000201E66B000E47
:102CE000E66EE66AE66EE66A740EE66EE66A85EC05
:102CF0002BF0146E060EE15E14506D92699468A478
:102D000002D06894FCD71200D9CFE6FFE1CFD9FFFB
:102D1000E65202012D0EF06FFD0EE71553E17E0E17
:102D2000E715E8407F0B040DF3CFC5F2F4CFC6F2F0
:102D3000000EC527040EC623C5C2C7F2C6C2C8F21C
:102D4000C775C5C2E9FFC6C2EAFFEF503C0BE842B7
:102D5000E8420D0835E1DF6A080EDF5C23E2C5C2F8
:102D6000E9FFC6C2EAFF020EE926000EEA22EE5093
:102D7000EFCFEAFFE96EEF50E66EDF50EA6A300F00
:102D8000E96E040EEA22E552E750EF6EC5C2E9FF94
:102D9000C6C2EAFF020EE926000EEA22EE2AEF2260
:102DA000DF2ADAD7C5C2E9FFC6C2EAFF020EE9266A
:102DB000000EEA22300EEE6E040EED6E0DD801D03C
:102DC0003AD805D0FD0EE715040801E15AD8E552BE
:102DD000E552E7CFD9FF12000201D56BF16BF46B1E
:102DE000F56BE96BD66BCFC2E9FFD0C2EAFFEF9E6D
:102DF000CF75CFC2E9FFD0C2EAFFEF9ECF75C7C241
:102E0000E9FFC8C2EAFFEF9ED96BDA6BDB6BDE6BC2
:102E1000DF6BE06B90D8000EE66EE66AE66EE66A5F
:102E2000030EE66EE66A85EC2BF0146E060EE15E8C
:102E300014508BEF1AF0020E0201D65D03E14EEC46
:102E40001BF01ED0D66BE9511AE1C7C2E9FFC8C218
:102E5000EAFFEE52080EEF6EC7C2E9FFC8C2EAFFF2
:102E6000020EE926000EEA22300EEE6E040EED6E22
:102E7000C7C2E9FFC8C2EAFF8C0EEF6E01D0E96B52
:102E80001200D9CFE6FFE1CFD9FFE652CFC2E9FF6A
:102E9000D0C2EAFFEF50400B01E0010EDF6E0201ED
:102EA000CF75080EC25D09E132C46EFF6E5003E0BB
:102EB000100EC26F02D0040EC26FD60528E1CFC239
:102EC000E9FFD0C2EAFF020EE926000EEA22380E20
:102ED000EE6E040EED6E80DB020E0201D55D07E1A1
:102EE000CFC2E9FFD0C2EAFF840EEF6E0FD0DF50F1
:102EF00007E1CFC2E9FFD0C2EAFFC80EEF6E06D0ED
:102F0000CFC2E9FFD0C2EAFF880EEF6E0FD0DEAF6E
:102F10000CD0E151E21107E005D0E2C2FAFF020154
:102F2000E151F96EFADF0201DE9FD66BE552E55200
:102F3000E7CFD9FF120004013051600BE842E842AC
:102F4000E842E842E842000901E059D031510C0A58
:102F500055E00B0A44E00C0A36E0010A27E00B0AB0
:102F600023E0020A21E0030A1DE0080A11E0010A39
:102F70000CE00F0A08E0030A01E040D00201D98FFB
:102F8000080EC26F3CD006DA3AD0EEEC1BF037D018
:102F90000201C30ED76F020ED86FD981010EDA6F0E
:102FA000D98F2DD057DA2BD02BD829D0345102010C
:102FB000D76FD86BC40ED727020ED823D981010E44
:102FC000DA6FD98F1CD00201D98F04013451EA6A1B
:102FD000C40FE96E020EEA2232C4EFFF10D0000ED9
:102FE000E66EE66AE66EE66A020EE66EE66A85EC74
:102FF0002BF0146E060EE15E145001D000D01200CA
:10300000D9CFE6FFE1CFD9FF030EE1260401320557
:1030100010E130511F0B00090CE10201D98F030EA2
:103020000401315D04E10201010EE56F02D00201ED
:10303000E56B0401325101E012D130511F0B02083F
:1030400001E00DD134510F0B000901E108D13451D9
:103050000F0B020801E203D1200E0201C25D01E064
:10306000FED0D98F040134BF1AD034510F0BE96E52
:10307000EA6AD890E936EA36C90EE926020EEA2253
:10308000EECFDEFFEDCFDDFF34510F0BEA6AED0F1F
:10309000E96E020EEA22020EEFCFDBFF19D03451A7
:1030A0000F0BE96EEA6AD890E936EA36CF0EE926C8
:1030B000020EEA22EECFDEFFEDCFDDFF34510F0B23
:1030C000EA6AEA0FE96E020EEA22020EEFCFDBFF98
:1030D000D950020FE96EDACFEAFFEF50010B03E19E
:1030E000000EDF9401D0DF8434BF10D034510F0BB9
:1030F000E96EEA6AD890E936EA36C90EE926020E88
:10310000EA22DECFEEFFDDCFEDFF0FD034510F0B03
:10311000E96EEA6AD890E936EA36CF0EE926020E61
:10312000EA22DECFEEFFDDCFEDFF030E315D23E1BE
:10313000DECFE9FFDDCFEAFFEF50800B13E034BFB5
:1031400009D034510F0BEA6AED0FE96E020EEA2244
:10315000EF8208D034510F0BEA6AEA0FE96E020ED3
:10316000EA22EF82840E146EDECFE9FFDDCFEAFFA4
:103170001450EF1274D0DF74DECFE9FFDDCFEAFF29
:10318000EF50800B1BE0DECFE9FFDDCFEAFFEF9EC3
:10319000DECFE9FFDDCFEAFFEF8C020EE66EE66AD6
:1031A000DECFE6FFDDCFE6FF050EE66EE66A85ECD4
:1031B0002BF0146E060EE15E145005D0DECFE9FF51
:1031C000DDCFEAFFEF8CDF74D950020FE96EDACF62
:1031D000EAFFEF50020B0EE1DECFE9FFDDCFEAFFA1
:1031E000EF50800B34E0DECFE9FFDDCFEAFFEF5098
:1031F000040B2DE1040134BF09D034510F0BEA6AEE
:10320000ED0FE96E020EEA22EF9208D034510F0B57
:10321000EA6AEA0FE96E020EEA22EF923B0E146EA2
:10322000DECFE9FFDDCFEAFF1450EF16020EE66EA7
:10323000E66ADECFE6FFDDCFE6FF050EE66EE66A64
:1032400085EC2BF0146E060EE15E145008D03B0E98
:10325000146EDECFE9FFDDCFEAFF1450EF16030E48
:10326000E15C02E2E16AE552E16EE552E7CFD9FFA7
:1032700012000201F2514DE1010EF26FF35149E1EA
:10328000010EF36F020ED65D0DE1CFC2E9FFD0C291
:10329000EAFFEE52EF6ACFC2E9FFD0C2EAFFC80EE2
:1032A000EF6E37D0D60535E1E96BC5C2E9FFC6C27E
:1032B000EAFFEE52080EEF6EC5C2E9FFC6C2EAFF92
:1032C000020EE926000EEA22300EEE6E040EED6EBE
:1032D000C5C2E9FFC6C2EAFF840EEF6E010EE96FB8
:1032E000C7C2E9FFC8C2EAFFEE52080EEF6EC7C2BE
:1032F000E9FFC8C2EAFF020EE926000EEA22300EFC
:10330000EE6E040EED6EC7C2E9FFC8C2EAFF800E82
:10331000EF6E12000201F46BF56B020ED65D1AE13E
:10332000C7C2E9FFC8C2EAFFEE52080EEF6EC7C27D
:10333000E9FFC8C2EAFF020EE926000EEA22380EB3
:10334000EE6E040EED6EC7C2E9FFC8C2EAFFC80EFA
:10335000EF6E1FD0DA510401365D0201DB5104012A
:10336000375904E236C4DAF237C4DBF235D9CFC2BA
:10337000E9FFD0C2EAFF020EE926000EEA22380E6B
:10338000EE6E040EED6ECFC2E9FFD0C2EAFFC80EAA
:10339000EF6E1200800E0401305D5BE10201C00E91
:1033A000D96F04013351030A34E0010A0EE0030A25
:1033B00003E00201D96B4DD00201460ED76F5D0EBE
:1033C000D86F120EDA6FDB6B44D03251F66EF76AAB
:1033D000D890F636F736070EF6265E0EF72209006D
:1033E000F5CFD7F20A00F5CFD8F2020E0201F76A44
:1033F000D725F66ED851F7220800F5CFDAF2030E82
:10340000F76AD725F66ED851F7220800F5CFDBF220
:1034100020D0030E325D1AE23251F66EF76AD89070
:10342000F636F736090EF6265E0EF7220900F5CFBE
:10343000D7F20A00F5CFD8F2D7C2F6FFD8C2F7FF0D
:103440000800F5500201DA6FDB6B02D00201D96B84
:1034500000D01200D9CFE6FFE1CFD9FF020EE1265E
:103460000401386B396B30511F0B020A12E0030A5A
:103470000DE0010A01E03BD00201D98F040138813F
:103480000201E50502E10401388331D00201D98F40
:103490002ED00201D98F040134BF10D034510F0B4C
:1034A000E96EEA6AD890E936EA36C90EE926020ED4
:1034B000EA22EECFDEFFEDCFDDFF0FD034510F0B50
:1034C000E96EEA6AD890E936EA36CF0EE926020EAE
:1034D000EA22EECFDEFFEDCFDDFFDECFE9FFDDCF6D
:1034E000EAFFEF50040B02E0010E386F00D002013A
:1034F000D9AF07D0380ED76F040ED86FD981020E1E
:10350000DA6F020EE15C02E2E16AE552E16EE55239
:10351000E7CFD9FF12006D980201D9BF2BD0DEAFE3
:1035200009D0020ED66FF55101E1F4DE0201F36B12
:10353000F26B1FD0C7C2E9FFC8C2EAFFEE52080E05
:10354000EF6EC7C2E9FFC8C2EAFF020EE926000E0D
:10355000EA22300EEE6E040EED6EC7C2E9FFC8C25D
:10356000EAFF8C0EEF6ECFC2E9FFD0C2EAFF840EF5
:10357000EF6E31D0040130AF0DD00201010ED66FD5
:10358000F45101E1C7DE0201F36BF26BF15101E18D
:1035900070DE21D00201020ED66FC7C2E9FFC8C299
:1035A000EAFFEE52080EEF6EC7C2E9FFC8C2EAFF9B
:1035B000020EE926000EEA22300EEE6E040EED6ECB
:1035C000C7C2E9FFC8C2EAFF840EEF6EF36BF26B6D
:1035D000F15101E14EDE1200D9CFE6FFE1CFD9FF74
:1035E000E652080EDF6E0201DA5D000EDB590BE2D7
:1035F000DAC2DFFFD55103E1010ED56F04D0D50546
:1036000002E1020ED56FDF50146E156A1450DA5DB8
:10361000DA6F1550DB59DB6FCFC2E9FFD0C2EAFF8A
:10362000EE52DFCFEFFF380EE36F040EE46FD9B137
:1036300019D0DF5016E0D7C2F6FFD8C2F7FFD72B5C
:10364000000ED8230800F550E66EE3C2E9FFE4C29D
:10365000EAFFE32B000EE423E552E750EF6EDF06AE
:10366000E8D717D0DF5015E0D7C2E9FFD8C2EAFF8C
:10367000D72B000ED823EF50E66EE3C2E9FFE4C279
:10368000EAFFE32B000EE423E552E750EF6EDF067E
:10369000E9D7E552E552E7CFD9FF1200D9CFE6FFCF
:1036A000E1CFD9FF020EE126C5C2E9FFC6C2EAFF9B
:1036B000EE52EFCFDFFFDFCF14F014500201DF5DD9
:1036C000000EE05902E2DFC2DFFFDF50146E156A20
:1036D0001450DF5DDF6F1550E059E06F010EDB6ABB
:1036E000DF50F36E010EDBCFF4FFF350F45C16E213
:1036F000010EDB50EA6A380FE96E040EEA22EF5041
:10370000E66EDCC2E9FFDDC2EAFFDC2B000EDD2342
:10371000E552E750EF6E010EDB2AE2D7000ED880AB
:10372000DF55000EE05528E2C7C2E9FFC8C2EAFF34
:10373000EE52080EEF6EC7C2E9FFC8C2EAFF020EE2
:10374000E926000EEA22380EEE6E040EED6EC5C2BA
:10375000E9FFC6C2EAFFEF50400B07E1C7C2E9FF2D
:10376000C8C2EAFFC80EEF6E06D0C7C2E9FFC8C2E2
:10377000EAFF880EEF6E28D0C7C2E9FFC8C2EAFF91
:10378000EE52080EEF6EC7C2E9FFC8C2EAFF020E92
:10379000E926000EEA22300EEE6E040EED6EC7C270
:1037A000E9FFC8C2EAFF840EEF6EE151E21107E0C3
:1037B00005D0E2C2FAFF0201E151F96EFADF02011F
:1037C000DE9FF15101E155DD020EE15C02E2E16AAA
:1037D000E552E16EE552E7CFD9FF1200D9CFE6FFFF
:1037E000E1CFD9FFE6520201D98F020EE66EE66AFA
:1037F000E66A710EE66E0F0EE66E82EC2FF0146E26
:10380000050EE15E1450DF6ADF50146E156A0C0E6F
:10381000145C000E155810E2DF50040DF3CFE9FFE1
:10382000F4CFEAFF000EE926040EEA22EE6AEE6A01
:10383000EE6AEE6ADF2AE8D76D8C010EE66EE66A64
:10384000E66AC40EE66E020EE66E82EC2FF0146E8F
:10385000050EE15E14506D9C0201080ECF6F040E40
:10386000D06F000EC56F040EC66FC5C2C7F2C6C2C8
:10387000C8F232C4C3F2C35103E1100EC26F13D0B9
:10388000010EE66EE66AC30EE66E020EE66E010EED
:10389000E66EE66A85EC2BF0146E060EE15E1450BF
:1038A0000201200EC26FE552E552E7CFD9FF1200A8
:1038B000D9CFE6FFE1CFD9FF020EE126000EDE6E82
:1038C000040EDD6EFD0EDB50E824166EFE0EDB509E
:1038D000040DF3501624040DF3CF14F0F4CF15F0BB
:1038E000D9CFE9FFDACFEAFF1450EE261550ED22CA
:1038F000DECFE9FFDDCFEAFFEF9EFD0EDB500FE1EB
:10390000FE0EEA6ADB34FE0BEA36E96EC90EE926E2
:10391000020EEA22DECFEEFFDDCFEDFF0ED0FE0E6F
:10392000EA6ADB34FE0BEA36E96ECF0EE926020EB8
:10393000EA22DECFEEFFDDCFEDFFDECFE9FFDDCF08
:10394000EAFFEF9CDECFE9FFDDCFEAFF040EE926B8
:10395000000EEA22EF8C020EE15C02E2E16AE5521F
:10396000E16EE552E7CFD9FF1200D9CFE6FFE1CFF4
:10397000D9FF020EE126FD0EDBA407D0E66AFE0E9B
:10398000DBCFE6FF95DFE552E552FD0EDBA208D066
:10399000010EE66EFE0EDBCFE6FF8ADFE552E55252
:1039A000FE0EDB50156A700F146E0F0E152214C038
:1039B000DEFF15C0DDFFDECFE9FFDDCFEAFFFD0E44
:1039C000DBCFEFFF020EE15C02E2E16AE552E16E5D
:1039D000E552E7CFD9FF1200D9CFE6FFE1CFD9FFFB
:1039E000020EE126FE0EDB5020E1C7C2E9FFC8C28D
:1039F000EAFFEE52080EEF6EC7C2E9FFC8C2EAFF47
:103A0000020EE926000EEA22300EEE6E040EED6E76
:103A1000C7C2E9FFC8C2EAFF8C0EEF6ECFC2E9FF52
:103A2000D0C2EAFF840EEF6E3DD0FD0EDB50E824DD
:103A3000166EFE0EDB50040DF3501624040DF3CF6A
:103A400014F0F4CF15F0000E1426040E152214C045
:103A5000DEFF15C0DDFF840E146EDECFE9FFDDCF83
:103A6000EAFF1450EF12FD0EDB50E824166EFE0E36
:103A7000DB50040DF3501624010F040DF3CF14F0A6
:103A8000F4CF15F0000E1426040E152214C0DEFF2C
:103A900015C0DDFF840E146EDECFE9FFDDCFEAFF37
:103AA0001450EF12020EE15C02E2E16AE552E16EAF
:103AB000E552E7CFD9FF1200D9CFE6FFE1CFD9FF1A
:103AC000020EE126FD0EDB500FE0FE0EEA6ADB344B
:103AD000FE0BEA36E96ECF0EE926020EEA22EECFA1
:103AE000DEFFEDCFDDFF0ED0FE0EEA6ADB34FE0B0B
:103AF000EA36E96EC90EE926020EEA22EECFDEFFB3
:103B0000EDCFDDFFD9CFE9FFDACFEAFFEE50ED10C0
:103B100003E1F36AF46A49D0DECFE9FFDDCFEAFFC3
:103B2000020EE926000EEA22FB0EDBCFEEFFFC0EB2
:103B3000DBCFEDFFDECFE9FFDDCFEAFFEE52FA0E7D
:103B4000DBCFEFFF400E146EDECFE9FFDDCFEAFFE3
:103B50001450EF16880E146EDECFE9FFDDCFEAFFBA
:103B60001450EF12FD0EDB500CE0FE0EEA6ADB345F
:103B7000FE0BEA36E96ECF0EE926020EEA22EF745A
:103B80000BD0FE0EEA6ADB34FE0BEA36E96EC90E94
:103B9000E926020EEA22EF74DECF14F0DDCF15F035
:103BA00014C0F3FF15C0F4FF00D0020EE15C02E286
:103BB000E16AE552E16EE552E7CFD9FF1200D9CFB5
:103BC000E6FFE1CFD9FF6DA84ED0FE0EEA6ADB34E6
:103BD000FE0BEA36E96ECF0EE926020EEA22EE501F
:103BE000EFCFEAFFE96E400EEE16EE6AEE6AEE6A7D
:103BF000FE0EEA6ADB34FE0BEA36E96ECF0EE926EA
:103C0000020EEA22EE50EFCFEAFFE96EEE7CFE0EE6
:103C1000EA6ADB34FE0BEA36E96ECF0EE926020EC5
:103C2000EA22EF74400E146EFE0EEA6ADB34FE0BDD
:103C3000EA36E96ECF0EE926020EEA22EE50EFCF09
:103C4000EAFFE96E1450EF16FE0EEA6ADB34FE0B53
:103C5000EA36E96ECF0EE926020EEA22EE50EFCFE9
:0E3C6000EAFFE96EEF7CE552E7CFD9FF1200D4
:023C6E009EAC0A
:103C700096D09E9CC3CF9FF0C4CFA0F00001995175
:103C800002E044EC24F0000188B525D09FC0E6FF97
:103C9000A0C0E6FFCEEC25F0E552E5520201300E61
:103CA0007F6F806F0001D5250201816F300E00010A
:103CB000D4250201826F300E0001D3250201836FEB
:103CC000300E0001D2250201846F3E0E856F000187
:103CD000030E956F64D00001A129EA6A8B0FE96E8B
:103CE000000EEA22EF50290803E0050EA15D32E341
:103CF000A1C092F0060E9203F3500001CC25000102
:103D0000936F93C0E6FF9251EA6A8B0FE96E000E43
:103D1000EA22EF50E66E9FC0E6FFA0C0E6FF49EC46
:103D200009F0E552E552E552E552050E00019325F2
:103D3000EA6A7F0FE96E020EEA223E0EEF6EE66A35
:103D4000CCEC08F0E5520001A16B030E956F000169
:103D5000899125D0A12BA1C0E6FFCCEC08F0E5525B
:103D6000C2820001A105926F060E9203F35000017A
:103D7000CC250001936F93C0E6FF9251EA6A8B0F46
:103D8000E96E000EEA22EF50E66E9FC0E6FFA0C08B
:103D9000E6FF49EC09F0E552E552E552E552120022
:103DA000D9CFE6FFE1CFD9FF070EE126DF6A010E8A
:103DB000DB6A020EDB6A00018AA11AD0050EDB6AFB
:103DC000060EDB6A050EDB2A060E01E3DB2A000E77
:103DD000D65C0EE3FF0ED75C0BE1050EDBCF14F0D3
:103DE000060EDBCF15F0E80E145C030E1558EAE35F
:103DF000F2A4AAD0F294030ED6CFDBFF040ED7CFE5
:103E0000DBFFDBCF16F016C017F0166A030EDB508F
:103E100000011610146E17C015F0010E14C0DBFF60
:103E2000020E15C0DBFFD950010FE96EDACFEAFFB1
:103E30000001AF51EE26B051ED22010EDBCF14F0A0
:103E4000020EDBCF15F015C014F0156A1450D76EB2
:103E5000010EDB50D66E00018AA176D08A7A540E0C
:103E6000616F626F300E636F720E646F8AA30FD042
:103E7000010EDF6E89810001CC6B00019A6BC36A71
:103E8000C46AE66ACCEC08F0E5529E9CC28200014E
:103E90008AA52CD0E66A410EE66E8050E66E63EC91
:103EA0000CF0E552E552E552060EE66E420EE66E65
:103EB0008150E66E63EC0CF0E552E552E5520C0ED3
:103EC000E66E430EE66E8250E66E63EC0CF0E55251
:103ED000E552E5520001120ECC6FDF5007E1CC6BCA
:103EE00002013E0E906F0001030E956F0001A55177
:103EF000A61118E000018AB705D00001A507000E41
:103F0000A65B0FD00001A951AA1104E0A907000E79
:103F1000AA5B07D0E80EA96F030EAA6FA507000ED3
:103F2000A65B07D0A551A61104E100018A918991F1
:103F30008A9A00018951040B07E00001A45104E1B1
:103F4000040EA46F966B976B070EE15C02E2E16AC8
:103F5000E552E16EE552E7CFD9FF120000018895E6
:103F600088918893410E625D03E0420E625D1EE11E
:103F7000630E645D09E163C0E6FF62C0E6FF91EC99
:103F800008F0E552E55211D0720E645D0EE10001B9
:103F9000630E956F966B976B63C0E6FF62C0E6FF9A
:103FA00091EC08F0E552E552C28234D0430E625DD6
:103FB0002BE14D0E635D28E1650E645D0EE13A0E66
:103FC000655D0BE188858A830001A16B01EC09F036
:103FD000E66ACCEC08F0E55216D0640E645D02E1AE
:103FE0008A9311D0720E645D0EE188850001CC6B5E
:103FF0000001A16B630E956F966B976BE66ACCEC34
:1040000008F0E552C28206D0540E625D03E1560EFE
:10401000635D00E1120012001200500E0001625DAB
:1040200032E1770E645D26E10001926B080E925D2D
:1040300020E2060E9225EA6A600FE96E000EEA227F
:10404000EF50780813E0060E9225EA6A600FE96ED9
:10405000000EEA22EF50E66E300E9225E66E63C047
:10406000E6FF71EC0AF0E552E552E5520001922BB1
:10407000DDD708D0720E645D05E163C0E6FFE7ECB2
:1040800009F0E552BAD0430E625D39E14D0E635D31
:1040900036E1650E645D02E18A8530D0640E645DB0
:1040A00002E18A952BD0720E645D28E1E66A410E2A
:1040B000E66E8050E66E63EC0CF0E552E552E55298
:1040C000060EE66E420EE66E8150E66E63EC0CF074
:1040D000E552E552E5520C0EE66E430EE66E825056
:1040E000E66E63EC0CF0E552E552E55202013E0E3D
:1040F000906F0001CC6B0001030E956F7ED0550EC2
:10410000625D10E1420E635D05E1650E645D02E1F2
:10411000F19E07D0420E635D04E1640E645D01E12F
:10412000F18E6BD04D0E625D68E1650E645D03E05B
:10413000640E645D09E164C0E6FF63C0E6FFE5EC80
:104140000CF0E552E55259D0660E645D1FE16B0E2E
:10415000695D1CE168C0E6FF67C0E6FF66C0E6FF78
:10416000300EE66EE66E2FEC25F0146E050EE15E65
:104170001450F3CF9DF0F4CF9EF09DC0E6FF9EC09B
:10418000E6FF72EC0DF0E552E55237D0720E645D39
:1041900034E169C0E6FF68C0E6FF67C0E6FF66C0BD
:1041A000E6FF300EE66E2FEC25F0146E050EE15E94
:1041B0001450F3CF9DF0F4CF9EF00001000ED88094
:1041C0009D55000E9E5503E29D2B000E9E239DC023
:1041D00014F09EC015F0166A176A14C0E6FF15C0E9
:1041E000E6FF16C0E6FF17C0E6FF63C0E6FF12EC6D
:1041F0000DF0186E050EE15E1850120064C0E6FF67
:1042000063C0E6FF62C0E6FF71EC0AF0E552E552DA
:10421000E5521200300E0001635D01E0B0D0700E77
:10422000645D06E166C0E6FF1FEC0EF0E552A6D025
:10423000640E645D08E18A91300EE66E1FEC0EF0AC
:10424000E5528A9A9BD0710E645D34E16AC0E6FF44
:1042500069C0E6FF68C0E6FF67C0E6FF66C0E6FF2C
:104260002FEC25F0146E050EE15E1450F3CF9DF097
:10427000F4CF9EF0176A186A010E196E9DC01AF0ED
:104280009EC01BF01C6A1A50175C146E1B50185805
:10429000156E1C501958166E14C0AFF015C0B0F052
:1042A000F294AFC0E6FFB0C0E6FFCFEC30F0E552CD
:1042B000E55264D0740E645D31E168C0E6FF67C00A
:1042C000E6FF66C0E6FF300EE66EE66E2FEC25F0E8
:1042D000146E050EE15E1450F3CF9DF0F4CF9EF006
:1042E00069C0E6FF9DC0E6FF9EC0E6FF6FEC0EF0E2
:1042F000E552E552E552F3CFAFF0F4CFB0F0000154
:104300000A0ED8809D55000E9E5505E30001898553
:104310000001A46B02D00001899530D0630E645D6A
:1043200025E169C0E6FF68C0E6FF67C0E6FF66C03A
:10433000E6FF300EE66E2FEC25F0146E050EE15E02
:104340001450F3CF9DF0F4CF9EF000019D519E11CB
:104350000CE09DC0A7F09EC0A8F0010EA75F000E64
:10436000A85BA7C0A5F0A8C0A6F008D0720E645D37
:1043700005E18A81A7C0A5F0A8C0A6F071D0310ED2
:10438000635D6EE1700E645D06E166C0E6FFF1EC10
:1043900010F0E55265D0640E645D06E1300EE66E05
:1043A000F1EC10F0E5525CD0720E645D34E16AC04D
:1043B000E6FF69C0E6FF68C0E6FF67C0E6FF66C0CB
:1043C000E6FF2FEC25F0146E050EE15E1450F3CFDE
:1043D0009DF0F4CF9EF0176A186A010E196E9DC009
:1043E0001AF09EC01BF01C6A1A50175C146E1B500A
:1043F0001858156E1C501958166E14C0B1F015C01F
:10440000B2F09E90B1C0E6FFB2C0E6FFB3EC30F070
:10441000E552E55225D0740E645D22E168C0E6FFE6
:1044200067C0E6FF66C0E6FF300EE66EE66E2FEC74
:1044300025F0146E050EE15E1450F3CF9DF0F4CF1D
:104440009EF069C0E6FF9DC0E6FF9EC0E6FF21EC3E
:1044500011F0E552E552E552F3CFB1F0F4CFB2F0EE
:1044600012004D0E0001625D1DE1440E635D1AE114
:10447000720E645D17E1310EE66E300EE66E760E5A
:10448000E66E320EE66E310EE66E500EE66E430EAE
:10449000E66E690EE66E09EC25F0146E080EE15E1C
:1044A000145066D0460E625D1CE1570E635D19E143
:1044B000720E645D16E1320EE66E330EE66E310E5C
:1044C000E66E300EE66EE66E320EE66E310EE66E8B
:1044D000300EE66E09EC25F0146E080EE15E145005
:1044E00047D0440E625D0FE1300E645D146E300EF5
:1044F000635D0A0DF35014240001996F9B6B9C6B54
:10450000010E956F35D0530E625D14E1490E635D67
:1045100011E1770E645D0EE19268CF0E936E9468A0
:104520000F0EC16E806A816A826A0001956B00017C
:10453000CE6B1ED0520E625D1BE14F0E635D18E123
:10454000520E645D15E169C0E6FF68C0E6FF67C012
:10455000E6FF66C0E6FF95EC28F0E552E552E5522D
:10456000E552F3CF9FF0F4CFA0F00001010E956F5C
:1045700012000001956BA36B0001CE6B00018A91C4
:104580008A938A9588918893889589918995000165
:10459000A46B12000201BD51EA6A3F0FE96E020EE0
:1045A000EA22EF50280852E10001946B0201BD514C
:1045B000EA6A3F0FE96E020EEA22EF50E66E000152
:1045C0009451EA6A600FE96E000EEA22E552E75064
:1045D000EF6E0201BD51EA6A3F0FE96E020EEA2258
:1045E000EF6A0001942B0201BD2B0201BC510201B4
:1045F000BD5D0DE2BD51EA6A3F0FE96E020EEA228F
:10460000EF50290804E0140E0001945DCFE302018D
:10461000BD51EA6A3F0FE96E020EEA22EF50E66EE4
:1046200000019451EA6A600FE96E000EEA22E55239
:10463000E750EF6E9451EA6A600FE96E000EEA22CD
:10464000EF50290803E10001010ECE6F12000001B6
:10465000CE052EE1000195512BE1000161515A0A6E
:1046600019E00E0A15E0060A11E0020A0DE0160A2A
:1046700009E0020A05E0050A01E00ED06FDC0CD06B
:10468000CADC0AD0C9DC08D0C8DC06D0B7DD04D04B
:10469000C1DD02D0E6DE00D00001955102E1F5EC6B
:1046A00012F00001955102E1010E956F0001606B5F
:1046B00012000001955102E1E6D070D095050EE19F
:1046C000956B0201BB51EA6A000FE96E010EEA2206
:1046D000230EEF6EBB2B0001CE6B60D0020E955DFA
:1046E00003E0030E955D5AE1A45101E0A407020E18
:1046F000955D03E1080E936F05D0030E955D02E111
:104700003C0E936F956B64C0E6FF63C0E6FF62C02A
:10471000E6FF61C0E6FF22EC08F0E552E552E55203
:10472000E5520001926B922B9251EA6A7F0FE96E7B
:10473000020EEA22EF503E0803E09351925DF3E34C
:104740009251E66EE66A7F0EE66E020EE66E02019A
:10475000BB51156A000F146E010E152214C0E6FF3E
:1047600015C0E6FF57EC2FF0166E060EE15E1650F0
:1047700000019251EA6A7F0FE96E020EEA22EF6AA7
:1047800092510201BB27BB51EA6A000FE96E010E8C
:10479000EA223E0EEF6EBB2B0001CE6B630E0001D2
:1047A000955D07E000018951010B03E10001A4516F
:1047B0000DE00001962B000E9723280E965D230E28
:1047C000975904E3966B976BCD0E956F9551146EC8
:1047D000156A153404E21450C808000E155453E24B
:1047E00095519F6FA06BC80E9F5F000EA05B9FC08E
:1047F000E6FFA0C0E6FFCEEC25F0E552E55202014F
:10480000BB51EA6A000FE96E010EEA223C0EEF6E20
:10481000BB29EA6A000FE96E010EEA225A0EEF6E1A
:10482000020EBB25EA6A000FE96E010EEA22450E70
:10483000EF6E300E0001D325E66E030E0201BB259C
:10484000EA6A000FE96E010EEA22E552E750EF6EC8
:10485000300E0001D225E66E040E0201BB25EA6A85
:10486000000FE96E010EEA22E552E750EF6E050EE9
:10487000BB25EA6A000FE96E010EEA223E0EEF6EDA
:10488000060EBB2776DE12000001990510E1E80E46
:104890009B5D030E9C5903E39B6B9C6B03D09B2B8E
:1048A000000E9C239BC09FF09CC0A0F020D0020E65
:1048B000995D07E177EC30F0F3CF9FF0F4CFA0F0F3
:1048C00016D0030E995D10E19A2B300E9A25E66EF4
:1048D0000201BB51EA6A000FE96E010EEA22E552BD
:1048E000E750EF6EBB2B03D0040E995D00E1120080
:1048F000D9CFE6FFE1CFD9FF040EE12600019F6B7F
:10490000A06BFF0EE66E010EE66E9FC014F0A0C015
:1049100015F0166A176A14C0E6FF15C0E6FF16C048
:10492000E6FF17C0E6FF13EC14F0186E060EE15E0A
:104930001850FFC1DFFF010E00C2DBFF0001200E97
:104940009F6F080EA06FFF0EE66E010EE66E9FC011
:1049500014F0A0C015F0166A176A14C0E6FF15C05F
:10496000E6FF16C0E6FF17C0E6FF13EC14F0186E62
:10497000060EE15E1850020EFFC1DBFF030E00C2FF
:10498000DBFFDF500DE1010EDB500AE1020EDB50D0
:10499000ED0806E1030EDB50100802E103D002D05F
:1049A0008A8AFFD7040EE15C02E2E16AE552E16E19
:0849B000E552E7CFD9FF120028
:0849B800D9CFE6FFE1CFD9FFE2
:1049C000FD0EDBCFE9FFFE0EDBCFEAFFEF501DE06F
:1049D000FD0EDBCFE9FFFE0EDBCFEAFFEF50E66E08
:1049E0000201BB51EA6A000FE96E010EEA22E552AC
:1049F000E750EF6EBB2BFD0EDBCFE9FFDB2AFE0E8F
:104A0000DBCFEAFF01E3DB2ADBD7E552E7CFD9FFB3
:104A10001200D9CFE6FFE1CFD9FFFE0EDBCF7FF248
:104A2000FD0EDBCF80F2FC0EDBCF81F2FB0EDBCF85
:104A300082F2FA0EDBCF83F2F90EDBCF84F2F80EAE
:104A4000DBCF85F2F70EDBCF86F202013E0E876FD9
:104A50000001020E956FE552E7CFD9FF1200D9CFC2
:104A6000E6FFE1CFD9FF020EE126DE6ADD6AFE0E27
:104A7000DBCF14F0156A14BE1568300E145E000EFC
:104A8000155A100E1502F3CF15F0270E1402F3502D
:104A90001526100E1402F3CF14F0F450152614C08E
:104AA000DEFF15C0DDFFFD0EDBCF14F0156A14BE6E
:104AB0001568300E145E000E155AE80E1502F3CF7D
:104AC00015F0030E1402F3501526E80E1402F3CF6E
:104AD00014F0F4501526D9CFE9FFDACFEAFF1450CD
:104AE000EE261550ED22FC0EDBCF14F0156A14BE35
:104AF0001568300E145E000E155A640E1502F3CFC1
:104B000015F01402F3CF14F0F4501526D9CFE9FFB5
:104B1000DACFEAFF1450EE261550ED22FB0EDBCF64
:104B200014F0156A14BE1568300E145E000E155A86
:104B30000A0E1502F3CF15F01402F3CF14F0F4505F
:104B40001526D9CFE9FFDACFEAFF1450EE2615502B
:104B5000ED22FA0EDBCF14F0156A14BE1568300E84
:104B6000145E000E155AD9CFE9FFDACFEAFF1450D0
:104B7000EE261550ED22DECF14F0DDCF15F014C077
:104B8000F3FF15C0F4FF020EE15C03E200D0E16A1E
:104B9000E552E16EE552E7CFD9FF1200D9CFE6FF2B
:104BA000E1CFD9FF0001D66BD56BD46BD36BD26B41
:104BB000D950FD0FE96EFF0EDA20EA6EEE50ED10CF
:104BC00001E1AFD2FD0EDBCF14F0FE0EDBCF15F00E
:104BD000D890155004E6E80E145C030E155812E345
:104BE000010ED56FFD0EDBCF14F0FE0EDBCF15F0FE
:104BF000E80E145E030E155AFD0E14C0DBFFFE0E08
:104C000015C0DBFFFD0EDBCF14F0FE0EDBCF15F081
:104C1000D890155004E6F40E145C010E155801E20C
:104C2000A5D0FD0EDBCF14F0FE0EDBCF15F0D89033
:104C3000155004E6840E145C030E155813E3090E98
:104C4000D46FFD0EDBCF14F0FE0EDBCF15F0840E1B
:104C5000145E030E155AFD0E14C0DBFFFE0E15C0C8
:104C6000DBFF83D0FD0EDBCF14F0FE0EDBCF15F0A3
:104C7000D890155004E6200E145C030E155813E36B
:104C8000080ED46FFD0EDBCF14F0FE0EDBCF15F057
:104C9000200E145E030E155AFD0E14C0DBFFFE0E2F
:104CA00015C0DBFF62D0FD0EDBCF14F0FE0EDBCFB4
:104CB00015F0D890155004E6BC0E145C020E155881
:104CC00013E3070ED46FFD0EDBCF14F0FE0EDBCF27
:104CD00015F0BC0E145E020E155AFD0E14C0DBFF5B
:104CE000FE0E15C0DBFF41D0FD0EDBCF14F0FE0E33
:104CF000DBCF15F0D890155004E6580E145C020E68
:104D0000155813E3060ED46FFD0EDBCF14F0FE0E24
:104D1000DBCF15F0580E145E020E155AFD0E14C0AE
:104D2000DBFFFE0E15C0DBFF20D0FD0EDBCF14F045
:104D3000FE0EDBCF15F0D890155004E6F40E145C8F
:104D4000010E155812E3050ED46FFD0EDBCF14F0E3
:104D5000FE0EDBCF15F0F40E145E010E155AFD0E9B
:104D600014C0DBFFFE0E15C0DBFF92D0FD0EDBCFC3
:104D700014F0FE0EDBCF15F0D890155004E6640E4B
:104D8000145C000E155801E283D0FD0EDBCF14F049
:104D9000FE0EDBCF15F0D890155004E6900E145C93
:104DA000010E155813E3040ED46FFD0EDBCF14F083
:104DB000FE0EDBCF15F0900E145E010E155AFD0E9F
:104DC00014C0DBFFFE0E15C0DBFF62D0FD0EDBCF93
:104DD00014F0FE0EDBCF15F0D890155004E62C0E23
:104DE000145C010E155813E3030ED46FFD0EDBCFD8
:104DF00014F0FE0EDBCF15F02C0E145E010E155ACA
:104E0000FD0E14C0DBFFFE0E15C0DBFF41D0FD0E12
:104E1000DBCF14F0FE0EDBCF15F0D890155004E672
:104E2000C80E145C000E155813E3020ED46FFD0E6D
:104E3000DBCF14F0FE0EDBCF15F0C80E145E000EB3
:104E4000155AFD0E14C0DBFFFE0E15C0DBFF20D08F
:104E5000FD0EDBCF14F0FE0EDBCF15F0D890155011
:104E600004E6640E145C000E155812E3010ED46FB4
:104E7000FD0EDBCF14F0FE0EDBCF15F0640E145EDA
:104E8000000E155AFD0E14C0DBFFFE0E15C0DBFF31
:104E9000FD0EDBCF14F0FE0EDBCF15F0D8901550D1
:104EA00004E6320E145C000E155801E2A5D0FD0E8A
:104EB000DBCF14F0FE0EDBCF15F0D890155004E6D2
:104EC0005A0E145C000E155813E3090ED36FFD0E35
:104ED000DBCF14F0FE0EDBCF15F05A0E145E000E81
:104EE000155AFD0E14C0DBFFFE0E15C0DBFF83D08C
:104EF000FD0EDBCF14F0FE0EDBCF15F0D890155071
:104F000004E6500E145C000E155813E3080ED36F20
:104F1000FD0EDBCF14F0FE0EDBCF15F0500E145E4D
:104F2000000E155AFD0E14C0DBFFFE0E15C0DBFF90
:104F300062D0FD0EDBCF14F0FE0EDBCF15F0D89063
:104F4000155004E6460E145C000E155813E3070EC8
:104F5000D36FFD0EDBCF14F0FE0EDBCF15F0460E47
:104F6000145E000E155AFD0E14C0DBFFFE0E15C0B8
:104F7000DBFF41D0FD0EDBCF14F0FE0EDBCF15F0D2
:104F8000D890155004E63C0E145C000E155813E33F
:104F9000060ED36FFD0EDBCF14F0FE0EDBCF15F047
:104FA0003C0E145E000E155AFD0E14C0DBFFFE0E03
:104FB00015C0DBFF20D0FD0EDBCF14F0FE0EDBCFE3
:104FC00015F0D890155004E6320E145C000E1558FA
:104FD00012E3050ED36FFD0EDBCF14F0FE0EDBCF18
:104FE00015F0320E145E000E155AFD0E14C0DBFFD4
:104FF000FE0E15C0DBFF92D0FD0EDBCF14F0FE0ECF
:10500000DBCF15F0D890155004E60A0E145C000EA4
:10501000155801E283D0FD0EDBCF14F0FE0EDBCF7E
:1050200015F0D890155004E6280E145C000E1558A3
:1050300013E3040ED36FFD0EDBCF14F0FE0EDBCFB7
:1050400015F0280E145E000E155AFD0E14C0DBFF7D
:10505000FE0E15C0DBFF62D0FD0EDBCF14F0FE0E9E
:10506000DBCF15F0D890155004E61E0E145C000E30
:10507000155813E3030ED36FFD0EDBCF14F0FE0EB5
:10508000DBCF15F01E0E145E000E155AFD0E14C077
:10509000DBFFFE0E15C0DBFF41D0FD0EDBCF14F0B1
:1050A000FE0EDBCF15F0D890155004E6140E145CFC
:1050B000000E155813E3020ED36FFD0EDBCF14F074
:1050C000FE0EDBCF15F0140E145E000E155AFD0E09
:1050D00014C0DBFFFE0E15C0DBFF20D0FD0EDBCFC2
:1050E00014F0FE0EDBCF15F0D890155004E60A0E32
:1050F000145C000E155812E3010ED36FFD0EDBCFCA
:1051000014F0FE0EDBCF15F00A0E145E000E155AD9
:10511000FD0E14C0DBFFFE0E15C0DBFFFD0EDBCF66
:10512000D2F0E552E7CFD9FF1200D9CFE6FFE1CFA9
:10513000D9FF0A0EE126FE0EDB5039080EE3FE0E03
:10514000DB50D00F146E156A14BE1568080E14C01B
:10515000DBFF090E15C0DBFF11D0FE0EDB50390856
:105160000DE2FE0EDB50C90F146E156A14BE1568F1
:10517000080E14C0DBFF090E15C0DBFF086A100E15
:10518000096E080EDBCF0DF0090EDBCF0EF085ECBB
:105190002EF0080E06C0DBFF090E07C0DBFFFD0E78
:1051A000DB5039080EE3FD0EDB50D00F146E156A8C
:1051B00014BE1568060E14C0DBFF070E15C0DBFF1A
:1051C00011D0FD0EDB5039080DE2FD0EDB50C90F8A
:1051D000146E156A14BE1568060E14C0DBFF070EA8
:1051E00015C0DBFF086A010E096E060EDBCF0DF05D
:1051F000070EDBCF0EF085EC2EF0060E06C0DBFFAF
:10520000070E07C0DBFFFC0EDB5039080EE3FC0E77
:10521000DB50D00F146E156A14BE1568040E14C04E
:10522000DBFF050E15C0DBFF11D0FC0EDB5039088B
:105230000DE2FC0EDB50C90F146E156A14BE156822
:10524000040E14C0DBFF050E15C0DBFF100E086E48
:10525000096A040EDBCF0DF0050EDBCF0EF085ECF6
:105260002EF0040E06C0DBFF050E07C0DBFFFB0EB1
:10527000DB5039080EE3FB0EDB50D00F146E156ABD
:1052800014BE1568020E14C0DBFF030E15C0DBFF51
:1052900011D0FB0EDB5039080DE2FB0EDB50C90FBD
:1052A000146E156A14BE1568020E14C0DBFF030EDF
:1052B00015C0DBFF060EDBCF1AF0070EDBCF1BF0AD
:1052C000080EDB501A24186E090EDB501B20196ED5
:1052D000040EDB501824166E050EDB501920176ED5
:1052E000020EDB501624146E030EDB501720156ED1
:1052F00014C0DEFF15C0DDFFDECF14F0DDCF15F0EA
:1053000014C0F3FF15C0F4FF0A0EE15C03E200D005
:0E531000E16AE552E16EE552E7CFD9FF1200E7
:02531E00DACFE4
:10532000E4FFE2CFDAFFE652E552E5CFDAFF110003
:10533000D8CFE4FFE0CFE4FFE46EDACFE4FFE2CFC2
:10534000DAFFE652E552E5CFDAFFE550E5CFE0FFC0
:10535000E5CFD8FF100011D8000189B102D072EC5E
:1053600015F0000189B105D005D927EC23F0D0EC68
:105370001EF037EC1EF0F0D712000F0EC11202D84B
:10538000E6EF14F0D9CFE6FFE1CFD9FFE652DF6AAE
:10539000DF50146E156AFF0E145C000E155809E2FA
:1053A000DF50EA6A000FE96E010EEA22EF6ADF2A97
:1053B000EFD70201BB6BBC6BBE6BBF6BCF0E9316FE
:1053C0009268936E9468C26A0F0EC16E960EC06E9C
:1053D000070EB46E806A816A826ADF6A080EDF5C3B
:1053E00009E2DF50EA6A7F0FE96E020EEA22EF6AF5
:1053F000DF2AF4D7B9EC22F078EC24F0E552E5523C
:10540000E7CFD9FF1200D9CFE6FFE1CFD9FFE652AF
:10541000938A939E240EAC6E900EAB6E710EAF6E9F
:10542000020EB06E080EB86EAE50DF6EE552E55259
:10543000E7CFD9FF1200D9CFE6FFE1CFD9FFFE0EAB
:10544000DB50AD6EE552E7CFD9FF1200D9CFE6FFB2
:10545000E1CFD9FF050EE126A00E0501001907E1F5
:10546000860E011904E1010E021901E1035116E152
:105470000001010ECD6F939681966D926D6ADF6A81
:10548000FF0EDF5C09E2E868E85004E0E80600D0BF
:1054900000D0FAD7DF2AF4D700EF00F0D880000E52
:1054A00005010055C20E0155010E0255000E0355AF
:1054B00001E241D000C5CFF501C5D0F502C5D1F557
:1054C00003C5D2F5186A1B0E196EB70E1A6E1B6A49
:1054D00018C006F019C007F01AC008F01BC009F088
:1054E000CFC50BF0D0C50CF0D1C50DF0D2C50EF074
:1054F00032EC30F006C014F007C015F008C016F00A
:1055000009C017F01406000E155A000E165A000EA8
:10551000175A010E14C0DBFF020E15C0DBFF030E8D
:1055200016C0DBFF040E17C0DBFF010EDB50AF6EB1
:10553000020EDB50B06E050EE15C02E2E16AE5525C
:10554000E16EE552E7CFD9FF1200D9CFE6FFE1CFF8
:10555000D9FFE652ABA205D0AB98AE50DF6EAB8858
:1055600002D0AE50DF6EDF5000D0E552E552E7CFFB
:10557000D9FF1200200E0201E76EC219E8AE02D078
:10558000E73402D0E750C25D03E36D50020B01E047
:105590004AD00001CF5115E1400EE66E3F0EE66E97
:1055A000020EE66E5BEC2CF0E552E552E55202018C
:1055B000BC6FBC51000805E20001010ECF6F020173
:1055C000BD6B0001CF5111E0AC50020B0EE0CE518B
:1055D0000CE10001955109E1CAEC22F00201BD2B5A
:1055E000BC51BD5D02E30001CF6B0001B45102E18B
:1055F00059EC23F00001B45114E10201BB51000841
:1056000010E20001A4510DE1BBC2E6FF000EE66E00
:10561000010EE66EBCEC2CF0E552E552E5520201BB
:10562000BB6B58EC2DF012000001D051D11104E1F8
:10563000100ED06F270ED16FD007000ED15B6DA278
:105640000AD0D051D11106E18A788AA802D08A8A7C
:1056500001D08A9A2ED00201C25103E18A988A9A17
:1056600028D0C20503E18A888A8A23D0020EC25D4F
:1056700003E18A888A9A1DD0040EC25D03E18A98EC
:105680008A8A17D0100EC25D07E10001D051D111F6
:1056900002E18A788A9A0DD0200EC25D0AE10001EB
:1056A000D051D11106E18A788AA802D08A9A01D015
:1056B0008A8A12001200120012001200D4EF2BF09E
:1056C000120027EF2CF00201E5051EE10201E605BC
:1056D0001BE1F1DF6D920201E66B0201100EC06F5B
:1056E0000E0EC16FC007000EC15BC051C111FAE1BF
:1056F0006D84080EC06F070EC16FC007000EC15B3E
:10570000C051C111FAE16D941200D9CFE6FFE1CF8B
:10571000D9FFFD0EDBCF08F0FE0EDBCF09F0050E42
:10572000081801E1095039E0E868081802E17F0E25
:10573000091831E0030E081801E109502AE0020EB1
:10574000081801E1095023E0010E081801E1095091
:105750001CE0740E081801E1095015E0750E0818D8
:1057600001E109500EE0730E081801E1095007E04D
:10577000720E081801E1095001E010D00FD09CDF33
:105780000DD098DF0BD097DF09D09BDF07D098DFD3
:1057900005D094DF03D091DF01D000D0010E00D0FE
:0857A000E552E7CFD9FF12002A
:0857A800040130511F0B010840
:1057B00001E04CD03051600BE842E842E842E84258
:1057C000E842010801E042D0345103E0340501E031
:1057D0003DD03151220A35E0030A28E0010A17E0E2
:1057E000210A0EE0010A01E031D00201C40ED76F98
:1057F000000ED86F080EDA6FDB6BD981D98F26D0F7
:105800000201C40ED76F000ED86FD98F1FD036C4D7
:10581000DFF237C4E0F20201000EDC6F050EDD6F2F
:105820004C0EE16F540EE26FDE8F10D00201CF0EEE
:10583000D76F050ED86F070EDA6FDB6BC10ED96F0D
:1058400005D032C4BFF00201D98F00D0120005018B
:10585000CF6B4B0ED06FD16BD26BD36BD46B080E6A
:10586000D56F0001B36B1A0EE66E010EE66EB5EC55
:105870001CF0E552E5521E0EE66E020EE66EB5EC29
:105880001CF0E552E552870EE66E080EE66E050E38
:10589000E66EE66A020EE66E5CEC1DF0146E050E16
:1058A000E15E1450F3CFBBF0F4CFBCF00001BD6B50
:1058B000BE6BB46B1200D9CFE6FFE1CFD9FF000178
:1058C000B36BBB51BC1102E1000E08D0BBC0E9FFB5
:1058D000BCC0EAFFEF50800B01E0010E000945E17A
:1058E000FC0EDBCF14F0BBC0E9FFBCC0EAFFEE52F8
:1058F000EF50D880145408E2BBC0E9FFBCC0EAFFF7
:10590000EE52FC0EEFCFDBFFB36BFC0EDB50B35D52
:1059100019E2B351EA6A080FE96E050EEA22EF5068
:10592000E66EB351E76EFD0EDBCFE9FFFE0EDBCF77
:10593000EAFFE750E926000EEA22E552E750EF6E53
:10594000B32BE3D7870EE66E080EE66E050EE66E05
:10595000E66A020EE66E5CEC1DF0146E050EE15E6A
:105960001450F3CFBBF0F4CFBCF00001B35100D022
:10597000E552E7CFD9FF1200D9CFE6FFE1CFD9FF3B
:105980000001B4510CE1FD0EDBCFB5F0FE0EDBCF14
:10599000B6F0FC0EDBCFB9F0010EBA6FB46FE55272
:1059A000E7CFD9FF1200D9CFE6FFE1CFD9FF030E31
:1059B000E1260001B45101E02ED0DF6AFD0EDBCFFD
:1059C00008F0FE0EDBCF09F0DE5208C0DEFF09C092
:1059D000DDFFDD52DF2ADF50146E156AFF0E14184A
:1059E00001E1155001E10BD0010EDBCFE9FFDB2A0D
:1059F000020EDBCFEAFF01E3DB2AEF50EBE1FD0E05
:105A0000DBCFB5F0FE0EDBCFB6F0DFCFB9F0000193
:105A1000010EBA6FB46F030EE15C02E2E16AE55277
:105A2000E16EE552E7CFD9FF1200D9CFE6FFE1CF13
:105A3000D9FF030EE1260001B45101E02FD0DF6A47
:105A4000FD0EDBCF08F0FE0EDBCF09F0DE5208C002
:105A5000DEFF09C0DDFFDD52DF2ADF50146E156A5C
:105A6000FF0E141801E1155001E10CD0010EDBCF3F
:105A7000F6FFDB2A020EDBCFF7FF01E3DB2A08008B
:105A8000F550EAE1FD0EDBCFB5F0FE0EDBCFB6F050
:105A9000DFCFB9F00001BA6B010EB46F030EE15C09
:105AA00002E2E16AE552E16EE552E7CFD9FF12006A
:105AB000D9CFE6FFE1CFD9FF020EE1260001BD51AB
:105AC000BE1102E1000E08D0BDC0E9FFBEC0EAFF72
:105AD000EF50800B01E0010E000901E085D0030EBC
:105AE000B45D01E1B46BB45101E17ED0020EB45D4E
:105AF00016E1E66A000EE66EE66A010EE66E020E3A
:105B0000E66E5CEC1DF0146E050EE15E1450F3CFF2
:105B1000BDF0F4CFBEF00001030EB46F65D0B40544
:105B200063E1400E146E156AB951145C000E1558ED
:105B300003E2400EDF6E02D0B9C0DFFFDF50B95D77
:105B4000B96F8F0EB76F050EB86F010EDFCFDBFF99
:105B5000BA5117E1010EDB5013E0B5C0F6FFB6C035
:105B6000F7FF0800F550B7C0E9FFB8C0EAFFEF6ED5
:105B7000B72B000EB823B52BB623010EDB06EAD7F0
:105B800015D0010EDB5012E0B5C0E9FFB6C0EAFF48
:105B9000EF50B7C0E9FFB8C0EAFFEF6EB72B000EB9
:105BA000B823B52BB623010EDB06EBD7B95108E1BC
:105BB000400EDF5C03E1020EB46F02D0030EB46F3F
:105BC000DFCFE6FF8F0EE66E050EE66E010EE66E87
:105BD000020EE66E5CEC1DF0146E050EE15E1450D4
:105BE000F3CFBDF0F4CFBEF0020EE15C02E2E16A59
:0C5BF000E552E16EE552E7CFD9FF12004C
:045BFC00006A0EAE7F
:105C000007EF2EF00D6C0E1EE86A0E22001E09AE84
:105C10000FEF2EF0086C091EE86A0922001E22EC24
:105C200031F009BE1FEF2EF000AE000C086C091E0B
:105C3000E86A0922046C051EE86A0522000C00BE11
:105C400016EF2EF00188FF0C006A0EAE2FEF2EF03B
:105C50000C6C0D1E0E1EE86A0D220E22001E09AEEF
:105C600039EF2EF0076C081E091EE86A0822092287
:105C7000001E96EC30F009BE4CEF2EF000AE000C8A
:105C8000076C081E091EE86A08220922036C041E1C
:105C9000051E04220522000C00BE40EF2EF00188F4
:105CA000FF0C006AE86A0EAE5EEF2EF00B6C0C1E65
:105CB0000D1E0E1E0C220D220E22001E09AE69EFD3
:105CC0002EF0066C071E081E091E07220822092254
:105CD000001E32EC30F009BE80EF2EF000AE000C5A
:105CE000066C071E081E091EE86A07220822092200
:105CF000026C031E041E051E032204220522000C52
:105D000000BE70EF2EF00188FF0C08C012F00850A2
:105D10000D02F4CF07F0F3CF06F009500E02F4CFD6
:105D200009F0F3CF08F00D02F3500726F4500822D3
:105D3000E86A092212500E02F3500726F450082296
:065D4000E86A0922000CD4
:0A5D46001201000202000008D80458
:105D50000A0000010102000109024300020100C023
:105D600032090400000102020100052400100104B0
:105D70002402020524060001052401000107058113
:105D80000308000209040100020A000000070502DE
:105D900002400000070582024000000403090434A9
:105DA00003690043006900720063007500690074B4
:105DB00000200054006500630068006E006F006CF6
:105DC000006F0067006900650073000000000000BC
:105DD000000000340369004300500031003200200D
:105DE0000062007900200050004900430063006910
:105DF00000720063007500690074002E0063006F7C
:0F5E0000006D0020000000585D9B5D9F5DD35D2D
:105E10002A0EF66E100EF76E000EF86E02010900E3
:105E2000F550FB6F0900F550FC6F03E1FB6701D0F3
:105E30003DD00900F550F66F0900F550F76F0900E5
:105E4000F550F86F09000900F550E96E0900F550AA
:105E5000EA6E090009000900F550F96F0900F550D4
:105E6000FA6F09000900F6CFFDF2F7CFFEF2F8CF86
:105E7000FFF2F6C2F6FFF7C2F7FFF8C2F8FF020121
:105E8000F95302E1FA5307E00900F550EE6EF90705
:105E9000F8E2FA07F9D7FDC2F6FFFEC2F7FFFFC22C
:0E5EA000F8FF0201FB07000EFC5BBFD71200EB
:025EAE00D9CF4A
:105EB000E6FFDACFE6FFFA0EE3CFD9FFFB0EE3CF22
:105EC000DAFFFC0EE3CFE9FFFD0EE3CFEAFFE9CFF7
:105ED000F3FFEACFF4FFF80EE35003E1F90EE350CD
:105EE00008E0F80EE30602E2F90EE306DECFEEFF6D
:105EF000F2D7FF0EE3CFDAFFE552FF0EE3CFD9FF73
:105F0000E5521200FE0EE3CFE9FFFF0EE3CFEAFFFA
:105F1000E9CFF3FFEACFF4FFFB0EE35003E1FC0E01
:105F2000E35009E0FB0EE30602E2FC0EE306FD0E81
:085F3000E350EE6EF1D7120000
:085F380006500B02F3CF02F04A
:105F4000F4CF03F00C02F3500326000EF420046E8D
:105F500006500D02F3500426000EF420056E065084
:105F60000E02F350052607500B02F3500326F4509F
:105F70000422000E052207500C02F3500426F450B0
:105F8000052207500D02F350052608500B02F3506E
:105F90000426F450052208500C02F350052609503F
:085FA0000B02F350052612006C
:085FA800D9CFE6FFDACFE6FFD6
:105FB000E1CFD9FFE2CFDAFFE652E652FC0EDBCFAB
:105FC00014F0FD0EDBCF15F0060ED8901436153602
:105FD000E804FBE114C0DEFF15C0DDFF010EDB505D
:105FE000BB6EDF50E840E8403F0B300B146ECF0E25
:105FF000BA141410BA6EE552E552E552E5CFDAFF55
:06600000E7CFD9FF1200FA
:0A600600D9CFE6FFDACFE6FFE1CFC5
:10601000D9FFE2CFDAFFE652E652FC0EDBCF14F0F6
:10602000FD0EDBCF15F0060ED89014361536E804B9
:10603000FBE114C0DEFF15C0DDFF010EDB50BE6EBC
:10604000DF50E840E8403F0B300B146ECF0EBD141C
:106050001410BD6EE552E552E552E5CFDAFFE7CF09
:04606000D9FF120052
:0C606400056A046A036A026A200EE76EF7
:10607000D890063607360836093602360336043617
:1060800005360B50025C0C5003580D5004580E504E
:10609000055809E30B50025E0C50035A0D50045A88
:0C60A0000E50055A062AE72EE4D7120025
:0460AC00D9CFE6FF63
:1060B000DACFE6FFE1CFD9FFE2CFDAFFFD0EDB500A
:1060C0007E0BCD6EFD0EDBAC02D0CD8E01D0CD9E11
:1060D000CF6ACE6A9E90DBAE02D09D8001D09D90AB
:0E60E000CD80E552E5CFDAFFE7CFD9FF120001
:0260EE00D9CF08
:1060F000E6FFDACFE6FFE1CFD9FFE2CFDAFFE652E3
:10610000E652D650DF6E010ED7CFDBFFDECF14F0A4
:10611000DDCF15F014C0F3FF15C0F4FFE552E552D2
:0C612000E552E5CFDAFFE7CFD9FF12000F
:04612C00056A046A92
:10613000036A180EE76ED89007360836093603361C
:10614000043605360C50035C0D5004580E500558AB
:1061500007E30C50035E0D50045A0E50055A072AEF
:06616000E72EEAD7120051
:0A616600D9CFE6FFDACFE6FFE1CF64
:10617000D9FFE2CFDAFFE652E652FC0EDBCFDEFFBC
:10618000DBCFDDFF010EDB50CF6EDF50CE6EE55270
:0E619000E552E552E5CFDAFFE7CFD9FF120066
:02619E00D9CF57
:1061A000E6FFDACFE6FFE1CFD9FFE2CFDAFFE65232
:1061B000E652FC0EDBCFDEFFDBCFDDFF010EDB5056
:1061C000D76EDF50D66EE552E552E552E5CFDAFFE5
:0661D000E7CFD9FF120029
:0A61D600D9CFE6FFDACFE6FFE1CFF4
:1061E000D9FFE2CFDAFFFD0EDB507F0BD56ED76A09
:1061F000D66AF294FD0EDBAE02D0F28A01D0F29A9A
:0E620000D58EE552E5CFDAFFE7CFD9FF1200C9
:02620E00D9CFE6
:10621000E6FFDACFE6FFE1CFD9FFE2CFDAFFFD0EEE
:10622000DB50FB0BCA6ECC6A9E92FD0EDBAE02D039
:106230009D8201D09D92CA84E552E5CFDAFFE7CF77
:04624000D9FF120070
:0C624400056A046A100EE76ED890083658
:106250000936043605360D50045C0E50055805E32A
:106260000D50045E0E50055A082AE72EF0D7120092
:10627000000EF36E00EE00F0080E01D81200EA6086
:1062800002D0EE6AFCD7F350E9601200EE6AFCD748
:1062900013EE00F023EE00F0F86A019C08EC2FF0FA
:0C62A0005CEC31F0ABEC29F0FBD71200F5
:0462AC00CD909D9064
:0262B0001200DA
:0662B200D59EF29A1200D5
:0262B8001200D2
:0662BA00000000000000DE
:1062C00000000000000000000000000000000000CE
:1062D00000000000000000000000000000000000BE
:0162E00000BD
:020000040030CA
:0100000024DB
:010001000EF0
:010002003FBE
:010003001EDE
:010005008179
:010006008178
:010008000FE8
:01000900C036
:01000A000FE6
:01000B00E014
:01000C000FE4
:01000D0040B2
:00000001FF
